:1000C0000000000000000000000000000000000030
:1000D0000000000000000000000000000000000020
:1000E0000000000000000000000000000000000010
:1000F0000000000000000000000000000000000000
:1001000000000000000000000000000000000000EF
:1001100000000000000000000000000000000000DF
:0401200000000000DB
:020000000BC330
:02000C00FECF25
:1000020001C001C0189518950EEF02BF4AD018958D
:10001200C598C498C198C49AC498C59AC59844E032
:10002200E5E7519168E0569510D06A95E1F74A9557
:10003200C1F788940AD009D008D007D006D005D0DD
:1000420004D003D0C59AC598089510F4C19A01C08E
:10005200C198C49AC4980895C29A4091610016D07A
:100062004091620013D04091630040680FD04091EC
:1000720064000CD04091650009D040916600406850
:1000820005D04091670002D0C298089518E0C09848
:10009200440F10F0C19801C0C19AC09A1A95B9F7DD
:1000A2000895C198C39AC398C19AC198C19A809978
:1000B20087C0C198C19A809944C08199ABC0C19848
:1000C200C19A80993EC0C198C19A80993DC08199D8
:1000D20093C0C198C19A809946C08199B7C0C1980E
:1000E200C19A80994FC0C198C19A80995AC081998A
:1000F2009FC0C198C19A8099C5C081996FC0C198AB
:10010200C19A8099B1C030918E00313019F430E03B
:1001120030938E0030918F00313019F430E03093FB
:100122008F0030919000313019F430E0309390001C
:1001320030919100313019F430E030939100C39A3C
:1001420008958ADFC39A089530918E00303049F4C1
:1001520031E030938E00309187004FEF3427309397
:100162008700CCD0EECF30918F00303049F431E0AF
:1001720030938F00309188004FEF342730938800FE
:10018200BDD0DFCF30919000303049F431E0309370
:100192009000309189004FEF342730938900AED020
:1001A200D0CF30919100303049F431E0309391005A
:1001B200309186004FEF3427309386009FD0C1CF15
:1001C200EDE6CAE802E3099300E0099300E009932F
:1001D20000E00993CAE888D191D0B3CFEDE6CAE82E
:1001E20002E3099300E0099300E0099300E0099318
:1001F200CAE88BD183D0A5CFEDE6CAE800EA09931D
:1002020006E8099301E0099300E00993CAE86CD17A
:1002120075D097CFEDE6CAE800EA099306E809939C
:1002220001E0099300E00993CAE86FD167D089CF52
:10023200EDE6CAE808EE099303E0099300E00993AA
:1002420000E00993CAE850D159D07BCFEDE6CAE865
:1002520008EE099303E0099300E0099300E0099393
:10026200CAE853D14BD06DCFEDE6CAE80AE0099354
:1002720000E0099300E0099300E00993CAE834D151
:100282003DD05FCFEDE6CAE80AE0099300E00993AA
:1002920000E0099300E00993CAE837D12FD051CF8B
:1002A2003327419151916191719188279927AA270A
:1002B200BB27CC27FF2730E2440F551F661F771F4D
:1002C200881F991FAA1FBB1FCC1F3A9559F4809310
:1002D200680090936900A0936A00B0936B00C0938A
:1002E2006C000895EDE1D291DD5FD3FDD083D08122
:1002F200D05DD7FDD083E831B1F7DECFCAE8EDE6B5
:10030200EAD0C9E7EAE801D110F001E001C000E05B
:100312000093850000918500013039F4C1E7EDE6D4
:10032200DAD0E1E7C9E7F1D006C0C1E7E9E7D3D007
:10033200E1E7CDE6EAD0E1E7CAE80FEF09930993D6
:1003420009930993CAE8ADE7F1D0EDE7CAE800E006
:10035200099301EE099305EF099305E00993CAE8B1
:10036200A5E70DD1009186000F3F11F4EDE601C023
:10037200E1E796DF58D0309187003F3F11F4C69AEB
:1003820001C0C698309188003F3F11F4C79A01C05E
:10039200C798309189003F3F11F4969A01C0969810
:1003A20037DE0895003011F40FE33CC0013011F440
:1003B20006E038C0023011F40BE534C0033011F40A
:1003C2000FE430C0043011F406E62CC0053011F4FD
:1003D2000DE628C0063011F40DE724C0073011F4F1
:1003E20007E020C0083011F40FE71CC0093011F4F7
:1003F2000FE618C00A3011F407E714C00B3011F4ED
:100402000CE710C00C3011F409E30CC00D3011F4EC
:100412000EE508C00E3011F409E704C00F3011F4E4
:1004220001E700C00895009168000F70BBDF0093E0
:1004320060000091680002950F70B4DF00936100C4
:10044200009169000F70AEDF0093620000916900B5
:1004520002950F70A7DF0093630000916A000F708E
:10046200A1DF0093640000916A0002950F709ADF89
:100472000093650000916B000F7094DF009366009B
:1004820000916B0002950F708DDF00936700009161
:1004920067000F33F9F400270093670000916600AC
:1004A2000F33C1F4002700936600009165000F33FB
:1004B20089F4002700936500009164000F3351F422
:1004C200002700936400009163000F3319F40027A2
:1004D2000093630008950191099301910993019199
:1004E200099301910993089531914191519161913B
:1004F200799189919991A991370F481F591F6A1FC4
:100502006293529342933293089531914191519162
:100512006191799189919991A991371B480B590B56
:100522006A0B629352934293329308950190119011
:10053200219031904990599069907990882499241A
:10054200AA24BB2430E2469457946794779420F40B
:10055200800C911CA21CB31CB794A7949794879407
:1005620077946794579447943A9589F74D925D92A0
:100572006D927D928D929D92AD92BD920895AF93B0
:100582000190119021903190419051906190719021
:1005920089909990A990B990CC24DD24EE24FF246F
:1005A200442755276627772788279927AA27BB1B21
:1005B20031E4001C111C221C331C441C551C661CFB
:1005C200771C3A9551F4AF910D921D922D923D9266
:1005D2004D925D926D927D920895441F551F661F44
:1005E200771F881F991FAA1FBB1F481959096A093B
:1005F2007B098C099D09AE09BF0950F4480D591DAC
:100602006A1D7B1D8C1D9D1DAE1DBF1D8894D1CF03
:100612000894CFCF0895F8940FED0DBF41E04093B9
:1006220060004DE6409361004FE34093620043EF68
:10063200409363004FE3409364004DEE40936500A6
:100642004EEE4093660000270093860000938700D9
:10065200009388000093890000938E0000938F001E
:10066200009390000093910005E003BF02E009BFF0
:1006720000E202BF00EC0BBF0FE005BF00E601BBCA
:1006820000E002BB0FEF07BB00E008BBD0E0F0E0E8
:10069200EDE600ED019302E6019306ED019300E021
:1006A2000193E9E704E901930BE901930FE7019351
:0806B20000E001937894FFCFF2
:00000001FF
